 getsysprops001

 Timestamp is 9b7e463c (reproducible build file hash)

 Preferred load address is 0000000180000000

 Start         Length     Name                   Class
 0001:00000000 00003440H .text$mn                CODE
 0001:00003440 00000036H .text$mn$00             CODE
 0001:00003476 00000092H .text$x                 CODE
 0002:00000000 000001c8H .idata$5                DATA
 0002:000001c8 00000038H .00cfg                  DATA
 0002:00000200 00000008H .CRT$XCA                DATA
 0002:00000208 00000008H .CRT$XCZ                DATA
 0002:00000210 00000008H .CRT$XIA                DATA
 0002:00000218 00000008H .CRT$XIC                DATA
 0002:00000220 00000008H .CRT$XIZ                DATA
 0002:00000228 00000008H .CRT$XLA                DATA
 0002:00000230 00000008H .CRT$XLZ                DATA
 0002:00000238 00000008H .CRT$XPA                DATA
 0002:00000240 00000008H .CRT$XPZ                DATA
 0002:00000248 00000008H .CRT$XTA                DATA
 0002:00000250 00000010H .CRT$XTZ                DATA
 0002:00000258 00000000H .gehcont$y              DATA
 0002:00000258 00000000H .gfids$y                DATA
 0002:00000260 00002020H .rdata                  DATA
 0002:00002280 00000000H .rdata$CastGuardVftablesA DATA
 0002:00002280 00000000H .rdata$CastGuardVftablesC DATA
 0002:00002280 00000028H .rdata$T                DATA
 0002:000022a8 000000e0H .rdata$voltmd           DATA
 0002:00002388 00000320H .rdata$zzzdbg           DATA
 0002:000026a8 00000008H .rtc$IAA                DATA
 0002:000026b0 00000008H .rtc$IZZ                DATA
 0002:000026b8 00000008H .rtc$TAA                DATA
 0002:000026c0 00000008H .rtc$TZZ                DATA
 0002:000026c8 00000004H .tls                    DATA
 0002:000026cc 00000004H .tls$                   DATA
 0002:000026d0 00000008H .tls$ZZZ                DATA
 0002:000026d8 00000338H .xdata                  DATA
 0002:00002a10 00000368H .edata                  DATA
 0002:00002d78 0000008cH .idata$2                DATA
 0002:00002e04 00000014H .idata$3                DATA
 0002:00002e18 000001c8H .idata$4                DATA
 0002:00002fe0 00000486H .idata$6                DATA
 0003:00000000 00000080H .data                   DATA
 0003:00000080 0001b238H .bss                    DATA
 0004:00000000 000003c0H .pdata                  DATA

  Address         Publics by Value              Rva+Base               Lib:Object

 0000:00000000       __AbsoluteZero             0000000000000000     <absolute>
 0000:00000000       ___safe_se_handler_count   0000000000000000     <absolute>
 0000:00000000       ___safe_se_handler_table   0000000000000000     <absolute>
 0000:00000000       __arm64x_extra_rfe_table   0000000000000000     <absolute>
 0000:00000000       __arm64x_extra_rfe_table_size 0000000000000000     <absolute>
 0000:00000000       __arm64x_native_entrypoint 0000000000000000     <absolute>
 0000:00000000       __arm64x_redirection_metadata 0000000000000000     <absolute>
 0000:00000000       __arm64x_redirection_metadata_count 0000000000000000     <absolute>
 0000:00000000       __dynamic_value_reloc_table 0000000000000000     <absolute>
 0000:00000000       __enclave_config           0000000000000000     <absolute>
 0000:00000000       __guard_check_icall_a64n_fptr 0000000000000000     <absolute>
 0000:00000000       __guard_eh_cont_count      0000000000000000     <absolute>
 0000:00000000       __guard_eh_cont_table      0000000000000000     <absolute>
 0000:00000000       __guard_fids_count         0000000000000000     <absolute>
 0000:00000000       __guard_fids_table         0000000000000000     <absolute>
 0000:00000000       __guard_iat_count          0000000000000000     <absolute>
 0000:00000000       __guard_iat_table          0000000000000000     <absolute>
 0000:00000000       __guard_longjmp_count      0000000000000000     <absolute>
 0000:00000000       __guard_longjmp_table      0000000000000000     <absolute>
 0000:00000000       __hybrid_auxiliary_iat     0000000000000000     <absolute>
 0000:00000000       __hybrid_auxiliary_iat_copy 0000000000000000     <absolute>
 0000:00000000       __hybrid_code_map          0000000000000000     <absolute>
 0000:00000000       __hybrid_code_map_count    0000000000000000     <absolute>
 0000:00000000       __x64_code_ranges_to_entry_points 0000000000000000     <absolute>
 0000:00000000       __x64_code_ranges_to_entry_points_count 0000000000000000     <absolute>
 0000:00000100       __guard_flags              0000000000000100     <absolute>
 0000:00000000       __ImageBase                0000000180000000     <linker-defined>
 0001:00000000       ?NewObject@JNIEnv_@@QEAAPEAV_jobject@@PEAV_jclass@@PEAU_jmethodID@@ZZ 0000000180001000 f i libgetsysprops001.obj
 0001:00000024       ?TranslateError@@YAPEBDW4jvmtiError@@@Z 0000000180001024 f   libgetsysprops001.obj
 0001:000002dc       ?nsk_jni_check_exception@@YAHPEAUJNIEnv_@@QEBDH@Z 00000001800012dc f   libgetsysprops001.obj
 0001:00000420       ?nsk_jni_lverify@@YAHHPEAUJNIEnv_@@HQEBDH1ZZ 0000000180001420 f   libgetsysprops001.obj
 0001:000004c0       Agent_Initialize           00000001800014c0 f   libgetsysprops001.obj
 0001:00000650       Agent_OnAttach             0000000180001650 f   libgetsysprops001.obj
 0001:00000650       Agent_OnLoad               0000000180001650 f   libgetsysprops001.obj
 0001:00000658       Java_nsk_jvmti_unit_FollowReferences_FollowRefObjects_addRefToVerify 0000000180001658 f   libgetsysprops001.obj
 0001:00000814       Java_nsk_jvmti_unit_FollowReferences_FollowRefObjects_getTag 0000000180001814 f   libgetsysprops001.obj
 0001:000008d0       Java_nsk_jvmti_unit_FollowReferences_FollowRefObjects_resetRefsToVerify 00000001800018d0 f   libgetsysprops001.obj
 0001:000008d8       Java_nsk_jvmti_unit_FollowReferences_FollowRefObjects_resetTags 00000001800018d8 f   libgetsysprops001.obj
 0001:0000091c       Java_nsk_jvmti_unit_FollowReferences_FollowRefObjects_setTag 000000018000191c f   libgetsysprops001.obj
 0001:00000b68       Java_nsk_share_jvmti_ArgumentHandler_getAgentOptionsString 0000000180001b68 f   libgetsysprops001.obj
 0001:00000c14       Java_nsk_share_jvmti_DebugeeClass_checkStatus 0000000180001c14 f   libgetsysprops001.obj
 0001:00000c9c       Java_nsk_share_jvmti_DebugeeClass_resetAgentData 0000000180001c9c f   libgetsysprops001.obj
 0001:00000cfc       Java_nsk_share_jvmti_RedefineAgent_agentStatus 0000000180001cfc f   libgetsysprops001.obj
 0001:00000d08       Java_nsk_share_jvmti_RedefineAgent_isRedefined 0000000180001d08 f   libgetsysprops001.obj
 0001:00000d14       Java_nsk_share_jvmti_RedefineAgent_redefineAttempted 0000000180001d14 f   libgetsysprops001.obj
 0001:00000d20       MA_checkStatus             0000000180001d20 f   libgetsysprops001.obj
 0001:00000dc4       __local_stdio_printf_options 0000000180001dc4 f i libgetsysprops001.obj
 0001:00001468       exitOnError                0000000180002468 f   libgetsysprops001.obj
 0001:0000151c       fprintf                    000000018000251c f i libgetsysprops001.obj
 0001:00001560       nsk_complain               0000000180002560 f   libgetsysprops001.obj
 0001:0000158c       nsk_jvmti_createJVMTIEnv   000000018000258c f   libgetsysprops001.obj
 0001:000016bc       nsk_jvmti_lverify          00000001800026bc f   libgetsysprops001.obj
 0001:000017ac       nsk_jvmti_parseOptions     00000001800027ac f   libgetsysprops001.obj
 0001:000019fc       nsk_jvmti_resetAgentData   00000001800029fc f   libgetsysprops001.obj
 0001:00001a70       nsk_jvmti_resumeSync       0000000180002a70 f   libgetsysprops001.obj
 0001:00001b14       nsk_jvmti_waitForSync      0000000180002b14 f   libgetsysprops001.obj
 0001:00001c18       nsk_lcomplain              0000000180002c18 f   libgetsysprops001.obj
 0001:00001c38       nsk_ldisplay               0000000180002c38 f   libgetsysprops001.obj
 0001:00001c58       nsk_ltrace                 0000000180002c58 f   libgetsysprops001.obj
 0001:00001c78       nsk_lvcomplain             0000000180002c78 f   libgetsysprops001.obj
 0001:00001e30       nsk_lvdisplay              0000000180002e30 f   libgetsysprops001.obj
 0001:00001e7c       nsk_lverify                0000000180002e7c f   libgetsysprops001.obj
 0001:00001ed8       nsk_lvtrace                0000000180002ed8 f   libgetsysprops001.obj
 0001:00001f38       nsk_printf                 0000000180002f38 f   libgetsysprops001.obj
 0001:00001f60       nsk_vprintf                0000000180002f60 f   libgetsysprops001.obj
 0001:00002014       printf                     0000000180003014 f i libgetsysprops001.obj
 0001:00002514       __raise_securityfailure    0000000180003514 f   MSVCRT:gs_report.obj
 0001:00002548       __report_gsfailure         0000000180003548 f   MSVCRT:gs_report.obj
 0001:00002788       __GSHandlerCheck           0000000180003788 f   MSVCRT:gshandler.obj
 0001:000027a8       __GSHandlerCheckCommon     00000001800037a8 f   MSVCRT:gshandler.obj
 0001:00002820       __security_check_cookie    0000000180003820 f   MSVCRT:amdsecgs.obj
 0001:00002b60       _DllMainCRTStartup         0000000180003b60 f   MSVCRT:dll_dllmain.obj
 0001:00002ba0       __scrt_acquire_startup_lock 0000000180003ba0 f   MSVCRT:utility.obj
 0001:00002bdc       __scrt_dllmain_after_initialize_c 0000000180003bdc f   MSVCRT:utility.obj
 0001:00002c10       __scrt_dllmain_before_initialize_c 0000000180003c10 f   MSVCRT:utility.obj
 0001:00002c28       __scrt_dllmain_crt_thread_attach 0000000180003c28 f   MSVCRT:utility.obj
 0001:00002c50       __scrt_dllmain_crt_thread_detach 0000000180003c50 f   MSVCRT:utility.obj
 0001:00002c68       __scrt_dllmain_exception_filter 0000000180003c68 f   MSVCRT:utility.obj
 0001:00002cc8       __scrt_dllmain_uninitialize_c 0000000180003cc8 f   MSVCRT:utility.obj
 0001:00002cf8       __scrt_dllmain_uninitialize_critical 0000000180003cf8 f   MSVCRT:utility.obj
 0001:00002d0c       __scrt_initialize_crt      0000000180003d0c f   MSVCRT:utility.obj
 0001:00002d58       __scrt_initialize_onexit_tables 0000000180003d58 f   MSVCRT:utility.obj
 0001:00002de4       __scrt_is_nonwritable_in_current_image 0000000180003de4 f   MSVCRT:utility.obj
 0001:00002e7c       __scrt_release_startup_lock 0000000180003e7c f   MSVCRT:utility.obj
 0001:00002ea0       __scrt_uninitialize_crt    0000000180003ea0 f   MSVCRT:utility.obj
 0001:00002ecc       _onexit                    0000000180003ecc f   MSVCRT:utility.obj
 0001:00002f08       atexit                     0000000180003f08 f   MSVCRT:utility.obj
 0001:00002f20       __crt_debugger_hook        0000000180003f20 f   MSVCRT:utility_desktop.obj
 0001:00002f28       __scrt_fastfail            0000000180003f28 f   MSVCRT:utility_desktop.obj
 0001:00003074       _guard_check_icall_nop     0000000180004074 f i MSVCRT:guard_support.obj
 0001:00003078       __security_init_cookie     0000000180004078 f   MSVCRT:gs_support.obj
 0001:00003124       DllMain                    0000000180004124 f   MSVCRT:dll_dllmain_stub.obj
 0001:00003148       ?__scrt_initialize_type_info@@YAXXZ 0000000180004148 f   MSVCRT:tncleanup.obj
 0001:00003158       ?__scrt_uninitialize_type_info@@YAXXZ 0000000180004158 f   MSVCRT:tncleanup.obj
 0001:00003164       __local_stdio_scanf_options 0000000180004164 f i MSVCRT:default_local_stdio_options.obj
 0001:0000316c       __scrt_initialize_default_local_stdio_options 000000018000416c f   MSVCRT:default_local_stdio_options.obj
 0001:00003188       __scrt_get_dyn_tls_init_callback 0000000180004188 f   MSVCRT:dyn_tls_init.obj
 0001:00003190       _RTC_Initialize            0000000180004190 f   MSVCRT:initsect.obj
 0001:000031cc       _RTC_Terminate             00000001800041cc f   MSVCRT:initsect.obj
 0001:00003208       __isa_available_init       0000000180004208 f   MSVCRT:cpu_disp.obj
 0001:000033b4       _get_startup_argv_mode     00000001800043b4 f   MSVCRT:argv_mode.obj
 0001:000033bc       __scrt_is_ucrt_dll_in_use  00000001800043bc f   MSVCRT:ucrt_detection.obj
 0001:000033d0       memcpy                     00000001800043d0 f   vcruntime:VCRUNTIME140.dll
 0001:000033d6       memset                     00000001800043d6 f   vcruntime:VCRUNTIME140.dll
 0001:000033dc       strchr                     00000001800043dc f   vcruntime:VCRUNTIME140.dll
 0001:000033e2       __C_specific_handler       00000001800043e2 f   vcruntime:VCRUNTIME140.dll
 0001:000033e8       __std_type_info_destroy_list 00000001800043e8 f   vcruntime:VCRUNTIME140.dll
 0001:000033ee       strcmp                     00000001800043ee f   ucrt:api-ms-win-crt-string-l1-1-0.dll
 0001:000033f4       strlen                     00000001800043f4 f   ucrt:api-ms-win-crt-string-l1-1-0.dll
 0001:000033fa       _initterm                  00000001800043fa f   ucrt:api-ms-win-crt-runtime-l1-1-0.dll
 0001:00003400       _initterm_e                0000000180004400 f   ucrt:api-ms-win-crt-runtime-l1-1-0.dll
 0001:00003406       _seh_filter_dll            0000000180004406 f   ucrt:api-ms-win-crt-runtime-l1-1-0.dll
 0001:0000340c       _configure_narrow_argv     000000018000440c f   ucrt:api-ms-win-crt-runtime-l1-1-0.dll
 0001:00003412       _initialize_narrow_environment 0000000180004412 f   ucrt:api-ms-win-crt-runtime-l1-1-0.dll
 0001:00003418       _initialize_onexit_table   0000000180004418 f   ucrt:api-ms-win-crt-runtime-l1-1-0.dll
 0001:0000341e       _register_onexit_function  000000018000441e f   ucrt:api-ms-win-crt-runtime-l1-1-0.dll
 0001:00003424       _execute_onexit_table      0000000180004424 f   ucrt:api-ms-win-crt-runtime-l1-1-0.dll
 0001:0000342a       _crt_atexit                000000018000442a f   ucrt:api-ms-win-crt-runtime-l1-1-0.dll
 0001:00003430       _cexit                     0000000180004430 f   ucrt:api-ms-win-crt-runtime-l1-1-0.dll
 0001:00003438       __acrt_initialize          0000000180004438 f   MSVCRT:ucrt_stubs.obj
 0001:00003438       __acrt_thread_attach       0000000180004438 f   MSVCRT:ucrt_stubs.obj
 0001:00003438       __acrt_thread_detach       0000000180004438 f   MSVCRT:ucrt_stubs.obj
 0001:00003438       __acrt_uninitialize        0000000180004438 f   MSVCRT:ucrt_stubs.obj
 0001:00003438       __acrt_uninitialize_critical 0000000180004438 f   MSVCRT:ucrt_stubs.obj
 0001:00003438       __scrt_stub_for_acrt_initialize 0000000180004438 f   MSVCRT:ucrt_stubs.obj
 0001:00003438       __scrt_stub_for_acrt_thread_attach 0000000180004438 f   MSVCRT:ucrt_stubs.obj
 0001:00003438       __scrt_stub_for_acrt_thread_detach 0000000180004438 f   MSVCRT:ucrt_stubs.obj
 0001:00003438       __scrt_stub_for_acrt_uninitialize 0000000180004438 f   MSVCRT:ucrt_stubs.obj
 0001:00003438       __scrt_stub_for_acrt_uninitialize_critical 0000000180004438 f   MSVCRT:ucrt_stubs.obj
 0001:00003438       __vcrt_initialize          0000000180004438 f   MSVCRT:ucrt_stubs.obj
 0001:00003438       __vcrt_thread_attach       0000000180004438 f   MSVCRT:ucrt_stubs.obj
 0001:00003438       __vcrt_thread_detach       0000000180004438 f   MSVCRT:ucrt_stubs.obj
 0001:00003438       __vcrt_uninitialize        0000000180004438 f   MSVCRT:ucrt_stubs.obj
 0001:00003438       __vcrt_uninitialize_critical 0000000180004438 f   MSVCRT:ucrt_stubs.obj
 0001:0000343c       __scrt_stub_for_is_c_termination_complete 000000018000443c f   MSVCRT:ucrt_stubs.obj
 0001:0000343c       _is_c_termination_complete 000000018000443c f   MSVCRT:ucrt_stubs.obj
 0001:00003450       _guard_dispatch_icall_nop  0000000180004450 f   MSVCRT:guard_dispatch.obj
 0001:00003470       _guard_xfg_dispatch_icall_nop 0000000180004470 f   MSVCRT:guard_xfg_dispatch.obj
 0002:00000000       __imp_RtlCaptureContext    0000000180005000     kernel32:KERNEL32.dll
 0002:00000008       __imp_RtlLookupFunctionEntry 0000000180005008     kernel32:KERNEL32.dll
 0002:00000010       __imp_RtlVirtualUnwind     0000000180005010     kernel32:KERNEL32.dll
 0002:00000018       __imp_UnhandledExceptionFilter 0000000180005018     kernel32:KERNEL32.dll
 0002:00000020       __imp_SetUnhandledExceptionFilter 0000000180005020     kernel32:KERNEL32.dll
 0002:00000028       __imp_GetCurrentProcess    0000000180005028     kernel32:KERNEL32.dll
 0002:00000030       __imp_TerminateProcess     0000000180005030     kernel32:KERNEL32.dll
 0002:00000038       __imp_IsProcessorFeaturePresent 0000000180005038     kernel32:KERNEL32.dll
 0002:00000040       __imp_CloseHandle          0000000180005040     kernel32:KERNEL32.dll
 0002:00000048       __imp_InitializeCriticalSectionAndSpinCount 0000000180005048     kernel32:KERNEL32.dll
 0002:00000050       __imp_DeleteCriticalSection 0000000180005050     kernel32:KERNEL32.dll
 0002:00000058       __imp_CreateEventW         0000000180005058     kernel32:KERNEL32.dll
 0002:00000060       __imp_GetModuleHandleW     0000000180005060     kernel32:KERNEL32.dll
 0002:00000068       __imp_GetProcAddress       0000000180005068     kernel32:KERNEL32.dll
 0002:00000070       __imp_IsDebuggerPresent    0000000180005070     kernel32:KERNEL32.dll
 0002:00000078       __imp_QueryPerformanceCounter 0000000180005078     kernel32:KERNEL32.dll
 0002:00000080       __imp_GetCurrentProcessId  0000000180005080     kernel32:KERNEL32.dll
 0002:00000088       __imp_GetCurrentThreadId   0000000180005088     kernel32:KERNEL32.dll
 0002:00000090       __imp_GetSystemTimeAsFileTime 0000000180005090     kernel32:KERNEL32.dll
 0002:00000098       __imp_DisableThreadLibraryCalls 0000000180005098     kernel32:KERNEL32.dll
 0002:000000a0       __imp_InitializeSListHead  00000001800050a0     kernel32:KERNEL32.dll
 0002:000000a8       \177KERNEL32_NULL_THUNK_DATA 00000001800050a8     kernel32:KERNEL32.dll
 0002:000000b0       __imp_memcpy               00000001800050b0     vcruntime:VCRUNTIME140.dll
 0002:000000b8       __imp_memset               00000001800050b8     vcruntime:VCRUNTIME140.dll
 0002:000000c0       __imp_strchr               00000001800050c0     vcruntime:VCRUNTIME140.dll
 0002:000000c8       __imp___C_specific_handler 00000001800050c8     vcruntime:VCRUNTIME140.dll
 0002:000000d0       __imp___std_type_info_destroy_list 00000001800050d0     vcruntime:VCRUNTIME140.dll
 0002:000000d8       \177VCRUNTIME140_NULL_THUNK_DATA 00000001800050d8     vcruntime:VCRUNTIME140.dll
 0002:000000e0       __imp_strtol               00000001800050e0     ucrt:api-ms-win-crt-convert-l1-1-0.dll
 0002:000000e8       \177api-ms-win-crt-convert-l1-1-0_NULL_THUNK_DATA 00000001800050e8     ucrt:api-ms-win-crt-convert-l1-1-0.dll
 0002:000000f0       __imp_malloc               00000001800050f0     ucrt:api-ms-win-crt-heap-l1-1-0.dll
 0002:000000f8       __imp_free                 00000001800050f8     ucrt:api-ms-win-crt-heap-l1-1-0.dll
 0002:00000100       \177api-ms-win-crt-heap-l1-1-0_NULL_THUNK_DATA 0000000180005100     ucrt:api-ms-win-crt-heap-l1-1-0.dll
 0002:00000108       __imp__errno               0000000180005108     ucrt:api-ms-win-crt-runtime-l1-1-0.dll
 0002:00000110       __imp_exit                 0000000180005110     ucrt:api-ms-win-crt-runtime-l1-1-0.dll
 0002:00000118       __imp__cexit               0000000180005118     ucrt:api-ms-win-crt-runtime-l1-1-0.dll
 0002:00000120       __imp__crt_atexit          0000000180005120     ucrt:api-ms-win-crt-runtime-l1-1-0.dll
 0002:00000128       __imp__execute_onexit_table 0000000180005128     ucrt:api-ms-win-crt-runtime-l1-1-0.dll
 0002:00000130       __imp__register_onexit_function 0000000180005130     ucrt:api-ms-win-crt-runtime-l1-1-0.dll
 0002:00000138       __imp__initialize_onexit_table 0000000180005138     ucrt:api-ms-win-crt-runtime-l1-1-0.dll
 0002:00000140       __imp__initialize_narrow_environment 0000000180005140     ucrt:api-ms-win-crt-runtime-l1-1-0.dll
 0002:00000148       __imp__configure_narrow_argv 0000000180005148     ucrt:api-ms-win-crt-runtime-l1-1-0.dll
 0002:00000150       __imp__seh_filter_dll      0000000180005150     ucrt:api-ms-win-crt-runtime-l1-1-0.dll
 0002:00000158       __imp__initterm_e          0000000180005158     ucrt:api-ms-win-crt-runtime-l1-1-0.dll
 0002:00000160       __imp__initterm            0000000180005160     ucrt:api-ms-win-crt-runtime-l1-1-0.dll
 0002:00000168       \177api-ms-win-crt-runtime-l1-1-0_NULL_THUNK_DATA 0000000180005168     ucrt:api-ms-win-crt-runtime-l1-1-0.dll
 0002:00000170       __imp___acrt_iob_func      0000000180005170     ucrt:api-ms-win-crt-stdio-l1-1-0.dll
 0002:00000178       __imp_fflush               0000000180005178     ucrt:api-ms-win-crt-stdio-l1-1-0.dll
 0002:00000180       __imp___stdio_common_vsprintf 0000000180005180     ucrt:api-ms-win-crt-stdio-l1-1-0.dll
 0002:00000188       __imp___stdio_common_vfprintf 0000000180005188     ucrt:api-ms-win-crt-stdio-l1-1-0.dll
 0002:00000190       \177api-ms-win-crt-stdio-l1-1-0_NULL_THUNK_DATA 0000000180005190     ucrt:api-ms-win-crt-stdio-l1-1-0.dll
 0002:00000198       __imp_strcmp               0000000180005198     ucrt:api-ms-win-crt-string-l1-1-0.dll
 0002:000001a0       __imp__strdup              00000001800051a0     ucrt:api-ms-win-crt-string-l1-1-0.dll
 0002:000001a0       __imp_strdup               00000001800051a0     ucrt:api-ms-win-crt-string-l1-1-0.dll
 0002:000001a8       __imp_strlen               00000001800051a8     ucrt:api-ms-win-crt-string-l1-1-0.dll
 0002:000001b0       __imp_strpbrk              00000001800051b0     ucrt:api-ms-win-crt-string-l1-1-0.dll
 0002:000001b8       __imp_strncpy              00000001800051b8     ucrt:api-ms-win-crt-string-l1-1-0.dll
 0002:000001c0       \177api-ms-win-crt-string-l1-1-0_NULL_THUNK_DATA 00000001800051c0     ucrt:api-ms-win-crt-string-l1-1-0.dll
 0002:000001c8       __guard_check_icall_fptr   00000001800051c8     MSVCRT:guard_support.obj
 0002:000001d0       __guard_xfg_check_icall_fptr 00000001800051d0     MSVCRT:guard_support.obj
 0002:000001d8       __guard_dispatch_icall_fptr 00000001800051d8     MSVCRT:guard_support.obj
 0002:000001e0       __guard_xfg_dispatch_icall_fptr 00000001800051e0     MSVCRT:guard_support.obj
 0002:000001e8       __guard_xfg_table_dispatch_icall_fptr 00000001800051e8     MSVCRT:guard_support.obj
 0002:000001f0       __castguard_check_failure_os_handled_fptr 00000001800051f0     MSVCRT:guard_support.obj
 0002:000001f8       __guard_memcpy_fptr        00000001800051f8     vcruntime:softmemtag.obj
 0002:00000200       __xc_a                     0000000180005200     MSVCRT:initializers.obj
 0002:00000208       __xc_z                     0000000180005208     MSVCRT:initializers.obj
 0002:00000210       __xi_a                     0000000180005210     MSVCRT:initializers.obj
 0002:00000220       __xi_z                     0000000180005220     MSVCRT:initializers.obj
 0002:00000228       __xl_a                     0000000180005228     MSVCRT:tlssup.obj
 0002:00000230       __xl_z                     0000000180005230     MSVCRT:tlssup.obj
 0002:00000238       __xp_a                     0000000180005238     MSVCRT:initializers.obj
 0002:00000240       __xp_z                     0000000180005240     MSVCRT:initializers.obj
 0002:00000248       __xt_a                     0000000180005248     MSVCRT:initializers.obj
 0002:00000250       __xt_z                     0000000180005250     MSVCRT:initializers.obj
 0002:00000260       g_refKindStr               0000000180005260     libgetsysprops001.obj
 0002:00000410       ??_C@_09BPLDFGCI@unknown_0@ 0000000180005410     libgetsysprops001.obj
 0002:00000420       ??_C@_0BL@FPNMECJD@JVMTI_HEAP_REFERENCE_CLASS@ 0000000180005420     libgetsysprops001.obj
 0002:00000440       ??_C@_0BL@FKGKKLNM@JVMTI_HEAP_REFERENCE_FIELD@ 0000000180005440     libgetsysprops001.obj
 0002:00000460       ??_C@_0CD@CAEHCFJF@JVMTI_HEAP_REFERENCE_ARRAY_ELEM@ 0000000180005460     libgetsysprops001.obj
 0002:00000488       ??_C@_0CC@DNEBMCNK@JVMTI_HEAP_REFERENCE_CLASS_LOAD@ 0000000180005488     libgetsysprops001.obj
 0002:000004b0       ??_C@_0BN@CJMIPEBB@JVMTI_HEAP_REFERENCE_SIGNERS@ 00000001800054b0     libgetsysprops001.obj
 0002:000004d0       ??_C@_0CH@HBOIDPEB@JVMTI_HEAP_REFERENCE_PROTECTION@ 00000001800054d0     libgetsysprops001.obj
 0002:000004f8       ??_C@_0BP@MDKGDGKL@JVMTI_HEAP_REFERENCE_INTERFACE@ 00000001800054f8     libgetsysprops001.obj
 0002:00000518       ??_C@_0CC@JJMIHNJH@JVMTI_HEAP_REFERENCE_STATIC_FIE@ 0000000180005518     libgetsysprops001.obj
 0002:00000540       ??_C@_0CD@IDHEEGID@JVMTI_HEAP_REFERENCE_CONSTANT_P@ 0000000180005540     libgetsysprops001.obj
 0002:00000568       ??_C@_0CA@EFFCHNG@JVMTI_HEAP_REFERENCE_SUPERCLASS@ 0000000180005568     libgetsysprops001.obj
 0002:00000588       ??_C@_0L@PCDFHGCJ@unknown_11@ 0000000180005588     libgetsysprops001.obj
 0002:00000598       ??_C@_0L@NJBICFOK@unknown_12@ 0000000180005598     libgetsysprops001.obj
 0002:000005a8       ??_C@_0L@MAADBEKL@unknown_13@ 00000001800055a8     libgetsysprops001.obj
 0002:000005b8       ??_C@_0L@IPECICGM@unknown_14@ 00000001800055b8     libgetsysprops001.obj
 0002:000005c8       ??_C@_0L@JGFJLDCN@unknown_15@ 00000001800055c8     libgetsysprops001.obj
 0002:000005d8       ??_C@_0L@LNHEOAOO@unknown_16@ 00000001800055d8     libgetsysprops001.obj
 0002:000005e8       ??_C@_0L@KEGPNBKP@unknown_17@ 00000001800055e8     libgetsysprops001.obj
 0002:000005f8       ??_C@_0L@CDPHMNGA@unknown_18@ 00000001800055f8     libgetsysprops001.obj
 0002:00000608       ??_C@_0L@DKOMPMCB@unknown_19@ 0000000180005608     libgetsysprops001.obj
 0002:00000618       ??_C@_0L@OJGIPJDB@unknown_20@ 0000000180005618     libgetsysprops001.obj
 0002:00000628       ??_C@_0CA@KAOFNDEM@JVMTI_HEAP_REFERENCE_JNI_GLOBAL@ 0000000180005628     libgetsysprops001.obj
 0002:00000648       ??_C@_0CC@HPFAJBK@JVMTI_HEAP_REFERENCE_SYSTEM_CLA@ 0000000180005648     libgetsysprops001.obj
 0002:00000670       ??_C@_0BN@FDEGFOHC@JVMTI_HEAP_REFERENCE_MONITOR@ 0000000180005670     libgetsysprops001.obj
 0002:00000690       ??_C@_0CB@HKIBCMAJ@JVMTI_HEAP_REFERENCE_STACK_LOCA@ 0000000180005690     libgetsysprops001.obj
 0002:000006b8       ??_C@_0BP@EAACMMOE@JVMTI_HEAP_REFERENCE_JNI_LOCAL@ 00000001800056b8     libgetsysprops001.obj
 0002:000006d8       ??_C@_0BM@IJDEOGOE@JVMTI_HEAP_REFERENCE_THREAD@ 00000001800056d8     libgetsysprops001.obj
 0002:000006f8       ??_C@_0BL@EDGPPKC@JVMTI_HEAP_REFERENCE_OTHER@ 00000001800056f8     libgetsysprops001.obj
 0002:00000714       ??_C@_04BCJPDBDA@Code@     0000000180005714     libgetsysprops001.obj
 0002:00000720       ??_C@_0BA@OCLMCFKC@LineNumberTable@ 0000000180005720     libgetsysprops001.obj
 0002:00000730       ??_C@_0BD@CPAEPILC@LocalVariableTable@ 0000000180005730     libgetsysprops001.obj
 0002:00000748       ??_C@_0BH@NMBDNHBD@LocalVariableTypeTable@ 0000000180005748     libgetsysprops001.obj
 0002:00000760       ??_C@_0O@HIHEEDNJ@StackMapTable@ 0000000180005760     libgetsysprops001.obj
 0002:00000770       ??_C@_0L@HCDIAMJG@?9?5?$CFs?0?5?$CFd?3?5@ 0000000180005770     libgetsysprops001.obj
 0002:00000780       ??_C@_0JI@HLPECLFI@?$CD?5?4?4?4?6?$CD?5ERROR?3?5too?5many?5complai@ 0000000180005780     libgetsysprops001.obj
 0002:00000820       ??_C@_0ED@JNEKCCOB@The?5following?5fake?5exception?5st@ 0000000180005820     libgetsysprops001.obj
 0002:00000868       ??_C@_0CN@FCNMDFBH@nsk?4share?4Fake_Exception_for_RU@ 0000000180005868     libgetsysprops001.obj
 0002:00000898       ??_C@_08PGFFNAEI@?$CI?$CFs?3?$CFd?$CJ?5@ 0000000180005898     libgetsysprops001.obj
 0002:000008a8       ??_C@_0DP@IENMAEGI@s?2test?2hotspot?2jtreg?2vmTestbase@ 00000001800058a8     libgetsysprops001.obj
 0002:000008e8       ??_C@_0BL@NDJLFFJB@?7at?5nsk_lvcomplain?$CI?$CFs?3?$CFd?$CJ?6@ 00000001800058e8     libgetsysprops001.obj
 0002:00000908       ??_C@_0BC@JOOKAFKF@?$CD?5ERROR?3?5?$CFs?0?5?$CFd?3?5@ 0000000180005908     libgetsysprops001.obj
 0002:00000920       ??_C@_09KJEAHMEH@?$CD?5ERROR?3?5@ 0000000180005920     libgetsysprops001.obj
 0002:0000092c       ??_C@_02GPIOPFAK@?$DO?$DO@ 000000018000592c     libgetsysprops001.obj
 0002:00000930       ??_C@_02FODMEDOG@?$DM?$DM@ 0000000180005930     libgetsysprops001.obj
 0002:00000934       ??_C@_02DJGKEECL@?4?4@     0000000180005934     libgetsysprops001.obj
 0002:00000938       ??_C@_0O@CJPGJOAF@?9?5?$CFs?0?5?$CFd?3?5?$CFs?5@ 0000000180005938     libgetsysprops001.obj
 0002:00000948       ??_C@_0CB@IAKPDOIC@?$CD?5?5?5verified?5assertion?5is?5FALSE@ 0000000180005948     libgetsysprops001.obj
 0002:00000970       ??_C@_0CO@LGONDEPD@stdout?3?5fflush?5failed?5?9?5err?$DN?$CFd?5@ 0000000180005970     libgetsysprops001.obj
 0002:000009a0       ??_C@_0CO@KBGKJPBD@stderr?3?5fflush?5failed?5?9?5err?$DN?$CFd?5@ 00000001800059a0     libgetsysprops001.obj
 0002:000009d0       ??_C@_06HPGEIPLA@?$DMnull?$DO@ 00000001800059d0     libgetsysprops001.obj
 0002:000009d8       ??_C@_0BB@JCNMKLLK@JVMTI_ERROR_NONE@ 00000001800059d8     libgetsysprops001.obj
 0002:000009f0       ??_C@_0BL@LDIMKLPH@JVMTI_ERROR_INVALID_THREAD@ 00000001800059f0     libgetsysprops001.obj
 0002:00000a10       ??_C@_0CB@PJFPAIKJ@JVMTI_ERROR_INVALID_THREAD_GROU@ 0000000180005a10     libgetsysprops001.obj
 0002:00000a38       ??_C@_0BN@LLMKHMNF@JVMTI_ERROR_INVALID_PRIORITY@ 0000000180005a38     libgetsysprops001.obj
 0002:00000a58       ??_C@_0CB@MBOFKAGB@JVMTI_ERROR_THREAD_NOT_SUSPENDE@ 0000000180005a58     libgetsysprops001.obj
 0002:00000a80       ??_C@_0BN@FABOLPBI@JVMTI_ERROR_THREAD_SUSPENDED@ 0000000180005a80     libgetsysprops001.obj
 0002:00000aa0       ??_C@_0BN@FDGNOBJM@JVMTI_ERROR_THREAD_NOT_ALIVE@ 0000000180005aa0     libgetsysprops001.obj
 0002:00000ac0       ??_C@_0BL@GOBIFKNJ@JVMTI_ERROR_INVALID_OBJECT@ 0000000180005ac0     libgetsysprops001.obj
 0002:00000ae0       ??_C@_0BK@FCMAJPPC@JVMTI_ERROR_INVALID_CLASS@ 0000000180005ae0     libgetsysprops001.obj
 0002:00000b00       ??_C@_0BP@IKLLBKEB@JVMTI_ERROR_CLASS_NOT_PREPARED@ 0000000180005b00     libgetsysprops001.obj
 0002:00000b20       ??_C@_0BN@KLPPLKG@JVMTI_ERROR_INVALID_METHODID@ 0000000180005b20     libgetsysprops001.obj
 0002:00000b40       ??_C@_0BN@BCEKOKND@JVMTI_ERROR_INVALID_LOCATION@ 0000000180005b40     libgetsysprops001.obj
 0002:00000b60       ??_C@_0BM@DFDGPME@JVMTI_ERROR_INVALID_FIELDID@ 0000000180005b60     libgetsysprops001.obj
 0002:00000b80       ??_C@_0BL@NELIEPEC@JVMTI_ERROR_NO_MORE_FRAMES@ 0000000180005b80     libgetsysprops001.obj
 0002:00000ba0       ??_C@_0BJ@BDBECFDM@JVMTI_ERROR_OPAQUE_FRAME@ 0000000180005ba0     libgetsysprops001.obj
 0002:00000bc0       ??_C@_0BK@MIIFNLOB@JVMTI_ERROR_TYPE_MISMATCH@ 0000000180005bc0     libgetsysprops001.obj
 0002:00000be0       ??_C@_0BJ@HPCAOILC@JVMTI_ERROR_INVALID_SLOT@ 0000000180005be0     libgetsysprops001.obj
 0002:00000c00       ??_C@_0BG@CHILOPNI@JVMTI_ERROR_DUPLICATE@ 0000000180005c00     libgetsysprops001.obj
 0002:00000c18       ??_C@_0BG@DIEMLHKM@JVMTI_ERROR_NOT_FOUND@ 0000000180005c18     libgetsysprops001.obj
 0002:00000c30       ??_C@_0BM@NHMCKHOB@JVMTI_ERROR_INVALID_MONITOR@ 0000000180005c30     libgetsysprops001.obj
 0002:00000c50       ??_C@_0BO@PPEDAJGL@JVMTI_ERROR_NOT_MONITOR_OWNER@ 0000000180005c50     libgetsysprops001.obj
 0002:00000c70       ??_C@_0BG@FCAIPEID@JVMTI_ERROR_INTERRUPT@ 0000000180005c70     libgetsysprops001.obj
 0002:00000c88       ??_C@_0CB@EGDBNKOI@JVMTI_ERROR_INVALID_CLASS_FORMA@ 0000000180005c88     libgetsysprops001.obj
 0002:00000cb0       ??_C@_0CG@DGKOGIAL@JVMTI_ERROR_CIRCULAR_CLASS_DEFI@ 0000000180005cb0     libgetsysprops001.obj
 0002:00000cd8       ??_C@_0BP@ICEALPKC@JVMTI_ERROR_FAILS_VERIFICATION@ 0000000180005cd8     libgetsysprops001.obj
 0002:00000cf8       ??_C@_0DC@JDACLMIO@JVMTI_ERROR_UNSUPPORTED_REDEFIN@ 0000000180005cf8     libgetsysprops001.obj
 0002:00000d30       ??_C@_0DE@GKDKNOMJ@JVMTI_ERROR_UNSUPPORTED_REDEFIN@ 0000000180005d30     libgetsysprops001.obj
 0002:00000d68       ??_C@_0BO@LAFKIOG@JVMTI_ERROR_INVALID_TYPESTATE@ 0000000180005d68     libgetsysprops001.obj
 0002:00000d88       ??_C@_0DH@INDGCLLB@JVMTI_ERROR_UNSUPPORTED_REDEFIN@ 0000000180005d88     libgetsysprops001.obj
 0002:00000dc0       ??_C@_0DE@NHEOMMGI@JVMTI_ERROR_UNSUPPORTED_REDEFIN@ 0000000180005dc0     libgetsysprops001.obj
 0002:00000df8       ??_C@_0CA@EKPNJOEP@JVMTI_ERROR_UNSUPPORTED_VERSION@ 0000000180005df8     libgetsysprops001.obj
 0002:00000e18       ??_C@_0BN@OFFMAHHL@JVMTI_ERROR_NAMES_DONT_MATCH@ 0000000180005e18     libgetsysprops001.obj
 0002:00000e38       ??_C@_0DN@HHBBLAKE@JVMTI_ERROR_UNSUPPORTED_REDEFIN@ 0000000180005e38     libgetsysprops001.obj
 0002:00000e78       ??_C@_0DO@HMBGBGNA@JVMTI_ERROR_UNSUPPORTED_REDEFIN@ 0000000180005e78     libgetsysprops001.obj
 0002:00000eb8       ??_C@_0BP@PBECGKHJ@JVMTI_ERROR_UNMODIFIABLE_CLASS@ 0000000180005eb8     libgetsysprops001.obj
 0002:00000ed8       ??_C@_0BK@CANILEHF@JVMTI_ERROR_NOT_AVAILABLE@ 0000000180005ed8     libgetsysprops001.obj
 0002:00000ef8       ??_C@_0CE@INJKMEFK@JVMTI_ERROR_MUST_POSSESS_CAPABI@ 0000000180005ef8     libgetsysprops001.obj
 0002:00000f20       ??_C@_0BJ@LBFPFPDM@JVMTI_ERROR_NULL_POINTER@ 0000000180005f20     libgetsysprops001.obj
 0002:00000f40       ??_C@_0BP@CHJPNNEM@JVMTI_ERROR_ABSENT_INFORMATION@ 0000000180005f40     libgetsysprops001.obj
 0002:00000f60       ??_C@_0BP@OMFMNLC@JVMTI_ERROR_INVALID_EVENT_TYPE@ 0000000180005f60     libgetsysprops001.obj
 0002:00000f80       ??_C@_0BN@BIBNPHHO@JVMTI_ERROR_ILLEGAL_ARGUMENT@ 0000000180005f80     libgetsysprops001.obj
 0002:00000fa0       ??_C@_0BK@KKNDHDCE@JVMTI_ERROR_NATIVE_METHOD@ 0000000180005fa0     libgetsysprops001.obj
 0002:00000fc0       ??_C@_0BK@PMKCFHAE@JVMTI_ERROR_OUT_OF_MEMORY@ 0000000180005fc0     libgetsysprops001.obj
 0002:00000fe0       ??_C@_0BK@NNJBDMNB@JVMTI_ERROR_ACCESS_DENIED@ 0000000180005fe0     libgetsysprops001.obj
 0002:00001000       ??_C@_0BI@GHECLMNC@JVMTI_ERROR_WRONG_PHASE@ 0000000180006000     libgetsysprops001.obj
 0002:00001018       ??_C@_0BF@OLIHJOII@JVMTI_ERROR_INTERNAL@ 0000000180006018     libgetsysprops001.obj
 0002:00001030       ??_C@_0BO@EOHGKJHI@JVMTI_ERROR_UNATTACHED_THREAD@ 0000000180006030     libgetsysprops001.obj
 0002:00001050       ??_C@_0CA@LKHFDACL@JVMTI_ERROR_INVALID_ENVIRONMENT@ 0000000180006050     libgetsysprops001.obj
 0002:00001070       ??_C@_0BA@MMFHLOKK@?$DMunknown?5error?$DO@ 0000000180006070     libgetsysprops001.obj
 0002:00001080       ??_C@_0CF@CBHOKDB@throwable?5?$DN?5jni?9?$DOExceptionOccur@ 0000000180006080     libgetsysprops001.obj
 0002:000010a8       ??_C@_03OFAPEBGM@?$CFs?6@  00000001800060a8     libgetsysprops001.obj
 0002:000010b0       ??_C@_0DM@LPIGEGNJ@s?2test?2hotspot?2jtreg?2vmTestbase@ 00000001800060b0     libgetsysprops001.obj
 0002:000010f0       ??_C@_0CC@NFCNPEPK@Exception?5in?5JNI?5call?5?$CIcleared?$CJ@ 00000001800060f0     libgetsysprops001.obj
 0002:00001118       ??_C@_0BJ@IBAKFIKF@jni?9?$DOExceptionDescribe?$CI?$CJ@ 0000000180006118     libgetsysprops001.obj
 0002:00001138       ??_C@_0BG@GGKALKMH@jni?9?$DOExceptionClear?$CI?$CJ@ 0000000180006138     libgetsysprops001.obj
 0002:00001150       ??_C@_0CF@JMGFGJLJ@?$CD?5?5?5verified?5JNI?5assertion?5is?5F@ 0000000180006150     libgetsysprops001.obj
 0002:00001178       ??_C@_07KBAMPNJK@verbose@  0000000180006178     libgetsysprops001.obj
 0002:00001180       ??_C@_0DN@PKJBOLAP@nsk_jvmti_parseOptions?$CI?$CJ?3?5unexp@ 0000000180006180     libgetsysprops001.obj
 0002:000011c0       ??_C@_05IMBNNINJ@trace@    00000001800061c0     libgetsysprops001.obj
 0002:000011c8       ??_C@_0DD@BJKGNDMB@nsk_jvmti_parseOptions?$CI?$CJ?3?5no?5va@ 00000001800061c8     libgetsysprops001.obj
 0002:000011fc       ??_C@_04CGFJFPFD@none@     00000001800061fc     libgetsysprops001.obj
 0002:00001204       ??_C@_06BMELKFMA@before@   0000000180006204     libgetsysprops001.obj
 0002:0000120c       ??_C@_05CMKPCFDK@after@    000000018000620c     libgetsysprops001.obj
 0002:00001214       ??_C@_03NFKEKGGK@all@      0000000180006214     libgetsysprops001.obj
 0002:00001218       ??_C@_0DM@NDNJGJKE@nsk_jvmti_parseOptions?$CI?$CJ?3?5uexpe@ 0000000180006218     libgetsysprops001.obj
 0002:00001258       ??_C@_08NBBJKJO@waittime@  0000000180006258     libgetsysprops001.obj
 0002:00001268       ??_C@_0DO@CMHGAOHC@nsk_jvmti_parseOptions?$CI?$CJ?3?5not?5i@ 0000000180006268     libgetsysprops001.obj
 0002:000012a8       ??_C@_0DL@LNMPBDLN@nsk_jvmti_parseOptions?$CI?$CJ?3?5negat@ 00000001800062a8     libgetsysprops001.obj
 0002:000012e8       ??_C@_0DA@GMFJNOJH@nsk_jvmti_parseOptions?$CI?$CJ?3?5unkno@ 00000001800062e8     libgetsysprops001.obj
 0002:00001318       ??_C@_0CO@CCIAMEAN@nsk_jvmti_parseOptions?$CI?$CJ?3?5found@ 0000000180006318     libgetsysprops001.obj
 0002:00001348       ??_C@_0CJ@OEGPCGDL@nsk_jvmti_parseOptions?$CI?$CJ?3?5out?5o@ 0000000180006348     libgetsysprops001.obj
 0002:00001378       ??_C@_0DI@NMBHPGGF@nsk_jvmti_parseOptions?$CI?$CJ?3?5too?5m@ 0000000180006378     libgetsysprops001.obj
 0002:000013b0       ??_C@_03POGCGECB@?5?0?$HO@ 00000001800063b0     libgetsysprops001.obj
 0002:000013b8       ??_C@_0CB@MLNJNCLJ@?5?5jvmti?5error?3?5code?$DN?$CFd?0?5name?$DN?$CFs@ 00000001800063b8     libgetsysprops001.obj
 0002:000013e0       ??_C@_0CD@OHBGDKMK@?$CD?5?5?5jvmti?5error?3?5code?$DN?$CFd?0?5name?$DN@ 00000001800063e0     libgetsysprops001.obj
 0002:00001408       ??_C@_0CG@JNNCGPHB@?$CD?5?5?5error?5expected?3?5code?$DN?$CFd?0?5na@ 0000000180006408     libgetsysprops001.obj
 0002:00001430       ??_C@_0EB@IMGKPCGE@?$CIstr_obj?5?$DN?5jni?9?$DONewStringUTF?$CIco@ 0000000180006430     libgetsysprops001.obj
 0002:00001480       ??_C@_0EA@HFOGGBCC@s?2test?2hotspot?2jtreg?2vmTestbase@ 0000000180006480     libgetsysprops001.obj
 0002:000014c0       ??_C@_05KKCIMGE@error@     00000001800064c0     libgetsysprops001.obj
 0002:000014c8       ??_C@_0BD@HGNAOMCP@agent_data_monitor@ 00000001800064c8     libgetsysprops001.obj
 0002:000014e0       ??_C@_0EB@OGCLGKLN@javaVM?9?$DOGetEnv?$CI?$CIvoid?5?$CK?$CK?$CJ?$CGjvmti_@ 00000001800064e0     libgetsysprops001.obj
 0002:00001530       ??_C@_0EA@PNBCDMOA@s?2test?2hotspot?2jtreg?2vmTestbase@ 0000000180006530     libgetsysprops001.obj
 0002:00001570       ??_C@_0CI@DDPIFBGM@init_agent_data?$CIjvmti_env?0?5?$CGage@ 0000000180006570     libgetsysprops001.obj
 0002:00001598       ??_C@_0DI@ILAHDLMP@?$CI?$CKagentThreadProc?$CJ?$CIjvmti_env?0?5a@ 0000000180006598     libgetsysprops001.obj
 0002:000015d0       ??_C@_0BD@KDBALNLB@JVMTI?5agent?5thread@ 00000001800065d0     libgetsysprops001.obj
 0002:000015e8       ??_C@_0BB@NOKBFPFO@java?1lang?1Thread@ 00000001800065e8     libgetsysprops001.obj
 0002:000015fc       ??_C@_06FALKBLGB@?$DMinit?$DO@ 00000001800065fc     libgetsysprops001.obj
 0002:00001608       ??_C@_0BG@IKDDPPGD@?$CILjava?1lang?1String?$DL?$CJV@ 0000000180006608     libgetsysprops001.obj
 0002:00001620       ??_C@_0EB@IFJBFEKC@?$CIthreadClass?5?$DN?5jni_env?9?$DOFindCla@ 0000000180006620     libgetsysprops001.obj
 0002:00001670       ??_C@_0GF@FGFIBKKL@?$CIthreadCtor?5?$DN?5jni_env?9?$DOGetMetho@ 0000000180006670     libgetsysprops001.obj
 0002:000016d8       ??_C@_0DN@NCPDJLOG@?$CIthreadName?5?$DN?5jni_env?9?$DONewStrin@ 00000001800066d8     libgetsysprops001.obj
 0002:00001720       ??_C@_0FE@PFKODBGC@?$CIthreadObject?5?$DN?5jni_env?9?$DONewObj@ 0000000180006720     libgetsysprops001.obj
 0002:00001780       ??_C@_0ED@HOBAHHJI@?$CIthreadGlobalRef?5?$DN?5jni_env?9?$DONew@ 0000000180006780     libgetsysprops001.obj
 0002:000017d0       ??_C@_0FN@HNJJAHFC@jvmti_env?9?$DORunAgentThread?$CIagent@ 00000001800067d0     libgetsysprops001.obj
 0002:00001830       ??_C@_0EA@MOJDNKDF@Debuggee?5status?5sync?5aborted?5be@ 0000000180006830     libgetsysprops001.obj
 0002:00001870       ??_C@_0CO@PGPGMHBJ@No?5status?5sync?5occured?5for?5time@ 0000000180006870     libgetsysprops001.obj
 0002:000018a0       ??_C@_0CL@DOEBDPKJ@Debuggee?5was?5not?5suspended?5on?5s@ 00000001800068a0     libgetsysprops001.obj
 0002:000018d0       ??_C@_0EA@EEOEJAEN@status?5?$DN?5syncDebuggeeStatus?$CIjni@ 00000001800068d0     libgetsysprops001.obj
 0002:00001910       ??_C@_0BL@JBCFNBMB@nsk_jvmti_resetAgentData?$CI?$CJ@ 0000000180006910     libgetsysprops001.obj
 0002:00001930       ??_C@_0EL@LPBEELIP@s?2test?2hotspot?2jtreg?2vmTestbase@ 0000000180006930     libgetsysprops001.obj
 0002:00001980       ??_C@_0CK@JDAMFDMJ@jvmti?9?$DOSetTag?$CIo?0?5tag?$CJ?5?$DN?$DN?5JVMTI_@ 0000000180006980     libgetsysprops001.obj
 0002:000019b0       ??_C@_0CC@DAMNHKNI@Can?8t?5set?5tag?5?$CFli?5for?5object?5?$CFl@ 00000001800069b0     libgetsysprops001.obj
 0002:000019d8       ??_C@_0DL@HAJPNKEF@jvmti?9?$DOGetObjectHashCode?$CIo?0?5?$CGha@ 00000001800069d8     libgetsysprops001.obj
 0002:00001a18       ??_C@_0BL@JFPIEOBF@Can?8t?5get?5hash?5object?5?$CFlx?6@ 0000000180006a18     libgetsysprops001.obj
 0002:00001a38       ??_C@_0BG@DICPHBKN@setTag?3?5?$CF08x?5?$DM?9?5?$CF?53li@ 0000000180006a38     libgetsysprops001.obj
 0002:00001a50       ??_C@_0DH@FCEEBDMJ@?$CIs?5?$DN?5jni?9?$DOGetStringUTFChars?$CIsIn@ 0000000180006a50     libgetsysprops001.obj
 0002:00001a88       ??_C@_0BJ@OKKGHDCN@Can?8t?5get?5string?5at?5?$CF?$CDp?6@ 0000000180006a88     libgetsysprops001.obj
 0002:00001aa8       ??_C@_0BP@EKFLGGFJ@Can?8t?5get?5string?5at?5?$CF?$CDp?3?5null?6@ 0000000180006aa8     libgetsysprops001.obj
 0002:00001ac8       ??_C@_06ICODBHCL@?5?1?1?5?$CFs@ 0000000180006ac8     libgetsysprops001.obj
 0002:00001ad0       ??_C@_0DB@KGFPLEGO@?$CIr?5?$DN?5jvmti?9?$DOGetTag?$CIo?0?5?$CGtag?$CJ?$CJ?5?$DN?$DN@ 0000000180006ad0     libgetsysprops001.obj
 0002:00001b08       ??_C@_0CO@PDAGBCGJ@Can?8t?5GetTag?5for?5object?5?$CFlx?4?5Re@ 0000000180006b08     libgetsysprops001.obj
 0002:00001b38       ??_C@_0CH@HPEODOHC@TEST_BUG?3?5Max?4?5number?5of?5refs?5r@ 0000000180006b38     libgetsysprops001.obj
 0002:00001b60       ??_C@_0DI@PHFCABIM@?$CIr?5?$DN?5jvmti?9?$DOGetTag?$CIfrom?0?5?$CGtagFr@ 0000000180006b60     libgetsysprops001.obj
 0002:00001b98       ??_C@_0DI@MDEGFNKD@TEST_BUG?3?5Can?8t?5GetTag?5for?5obje@ 0000000180006b98     libgetsysprops001.obj
 0002:00001bd0       ??_C@_0DE@MLELJAHM@?$CIr?5?$DN?5jvmti?9?$DOGetTag?$CIto?0?5?$CGtagTo?$CJ?$CJ@ 0000000180006bd0     libgetsysprops001.obj
 0002:00001c08       ??_C@_0BO@ONEFEOOD@Invoke?5GetSystemProperties?$CI?$CJ?6@ 0000000180006c08     libgetsysprops001.obj
 0002:00001c30       ??_C@_0GA@MBJFNMCI@s?2test?2hotspot?2jtreg?2vmTestbase@ 0000000180006c30     libgetsysprops001.obj
 0002:00001c90       ??_C@_0DA@KIJCDCDH@jvmti?9?$DOGetSystemProperties?$CI?$CGcou@ 0000000180006c90     libgetsysprops001.obj
 0002:00001cc0       ??_C@_0BK@MMCHCMAI@?5?5?5?5properties?5count?3?5?$CFd?6@ 0000000180006cc0     libgetsysprops001.obj
 0002:00001ce0       ??_C@_0BM@LBBKKCBE@?5?5?5?5properties?5list?3?5?50x?$CFp?6@ 0000000180006ce0     libgetsysprops001.obj
 0002:00001d00       ??_C@_0CA@MMAEPNNA@Check?5obtained?5properties?5list?6@ 0000000180006d00     libgetsysprops001.obj
 0002:00001d20       ??_C@_0EM@PCLELFIB@In?5?$CFs?5phase?5GetSystemProperties@ 0000000180006d20     libgetsysprops001.obj
 0002:00001d70       ??_C@_0FD@OCNOFBL@In?5?$CFs?5phase?5GetSystemProperties@ 0000000180006d70     libgetsysprops001.obj
 0002:00001dc8       ??_C@_0CE@NDPPHOF@Check?5each?5property?3?5?$CFd?5propert@ 0000000180006dc8     libgetsysprops001.obj
 0002:00001df0       ??_C@_0BI@NGOPABGM@?5?5?5?5property?5?$CD?$CFd?3?5?$FL?$CFs?$FN?6@ 0000000180006df0     libgetsysprops001.obj
 0002:00001e10       ??_C@_0EI@MFEKDEIA@In?5?$CFs?5phase?5GetSystemProperties@ 0000000180006e10     libgetsysprops001.obj
 0002:00001e58       ??_C@_0BM@NBAMMIGN@Deallocate?5properties?5list?6@ 0000000180006e58     libgetsysprops001.obj
 0002:00001e78       ??_C@_0CO@IDDPHEJA@jvmti?9?$DODeallocate?$CI?$CIunsigned?5cha@ 0000000180006e78     libgetsysprops001.obj
 0002:00001ea8       ??_C@_0BD@PFBGGHID@?5?5?4?4?4?5deallocated?6@ 0000000180006ea8     libgetsysprops001.obj
 0002:00001ec0       ??_C@_0CC@HCPFMLEK@Wait?5for?5debugee?5to?5become?5read@ 0000000180006ec0     libgetsysprops001.obj
 0002:00001ee8       ??_C@_0CL@IJEJJLCH@?$DO?$DO?$DO?5Check?5system?5properties?5in?5@ 0000000180006ee8     libgetsysprops001.obj
 0002:00001f14       ??_C@_04GLMHKBCH@live@     0000000180006f14     libgetsysprops001.obj
 0002:00001f20       ??_C@_0BH@HPEOJMHL@Let?5debugee?5to?5finish?6@ 0000000180006f20     libgetsysprops001.obj
 0002:00001f38       ??_C@_0CA@MNKGCBCG@nsk_jvmti_parseOptions?$CIoptions?$CJ@ 0000000180006f38     libgetsysprops001.obj
 0002:00001f58       ??_C@_0DN@MIAMNFPH@?$CIjvmti?5?$DN?5nsk_jvmti_createJVMTIE@ 0000000180006f58     libgetsysprops001.obj
 0002:00001f98       ??_C@_0CN@OIAPMHFE@?$DO?$DO?$DO?5Check?5system?5properties?5in?5@ 0000000180006f98     libgetsysprops001.obj
 0002:00001fc8       ??_C@_06FEOMBGJC@OnLoad@   0000000180006fc8     libgetsysprops001.obj
 0002:00001fd0       ??_C@_0CL@PIACJIPK@nsk_jvmti_setAgentProc?$CIagentPro@ 0000000180006fd0     libgetsysprops001.obj
 0002:00002010       ??_C@_1EC@JIJBPKFM@?$AAa?$AAp?$AAi?$AA?9?$AAm?$AAs?$AA?9?$AAw?$AAi?$AAn?$AA?9?$AAc?$AAo?$AAr?$AAe@ 0000000180007010     MSVCRT:thread_safe_statics.obj
 0002:00002058       ??_C@_1BK@MGMFAEKH@?$AAk?$AAe?$AAr?$AAn?$AAe?$AAl?$AA3?$AA2?$AA?4?$AAd?$AAl?$AAl@ 0000000180007058     MSVCRT:thread_safe_statics.obj
 0002:00002078       ??_C@_0BJ@JEBJOJFJ@SleepConditionVariableCS@ 0000000180007078     MSVCRT:thread_safe_statics.obj
 0002:00002098       ??_C@_0BJ@PGPPEPCC@WakeAllConditionVariable@ 0000000180007098     MSVCRT:thread_safe_statics.obj
 0002:000020b8       _pDefaultRawDllMain        00000001800070b8     MSVCRT:dll_dllmain.obj
 0002:000020b8       _pRawDllMain               00000001800070b8     MSVCRT:dll_dllmain.obj
 0002:000020c0       __xmm@ffffffffffffffffffffffffffffffff 00000001800070c0     MSVCRT:utility.obj
 0002:000020d0       _load_config_used          00000001800070d0     MSVCRT:loadcfg.obj
 0002:00002280       _tls_used                  0000000180007280     MSVCRT:tlssup.obj
 0002:000022a8       __volatile_metadata        00000001800072a8     <linker-defined>
 0002:000026a8       __rtc_iaa                  00000001800076a8     MSVCRT:initsect.obj
 0002:000026b0       __rtc_izz                  00000001800076b0     MSVCRT:initsect.obj
 0002:000026b8       __rtc_taa                  00000001800076b8     MSVCRT:initsect.obj
 0002:000026c0       __rtc_tzz                  00000001800076c0     MSVCRT:initsect.obj
 0002:000026c8       _tls_start                 00000001800076c8     MSVCRT:tlssup.obj
 0002:000026cc       _Init_thread_epoch         00000001800076cc     MSVCRT:thread_safe_statics.obj
 0002:000026d0       _tls_end                   00000001800076d0     MSVCRT:tlssup.obj
 0002:00002d78       __IMPORT_DESCRIPTOR_KERNEL32 0000000180007d78     kernel32:KERNEL32.dll
 0002:00002d8c       __IMPORT_DESCRIPTOR_VCRUNTIME140 0000000180007d8c     vcruntime:VCRUNTIME140.dll
 0002:00002da0       __IMPORT_DESCRIPTOR_api-ms-win-crt-heap-l1-1-0 0000000180007da0     ucrt:api-ms-win-crt-heap-l1-1-0.dll
 0002:00002db4       __IMPORT_DESCRIPTOR_api-ms-win-crt-runtime-l1-1-0 0000000180007db4     ucrt:api-ms-win-crt-runtime-l1-1-0.dll
 0002:00002dc8       __IMPORT_DESCRIPTOR_api-ms-win-crt-convert-l1-1-0 0000000180007dc8     ucrt:api-ms-win-crt-convert-l1-1-0.dll
 0002:00002ddc       __IMPORT_DESCRIPTOR_api-ms-win-crt-stdio-l1-1-0 0000000180007ddc     ucrt:api-ms-win-crt-stdio-l1-1-0.dll
 0002:00002df0       __IMPORT_DESCRIPTOR_api-ms-win-crt-string-l1-1-0 0000000180007df0     ucrt:api-ms-win-crt-string-l1-1-0.dll
 0002:00002e04       __NULL_IMPORT_DESCRIPTOR   0000000180007e04     kernel32:KERNEL32.dll
 0003:00000030       _Init_global_epoch         0000000180009030     MSVCRT:thread_safe_statics.obj
 0003:00000040       __security_cookie          0000000180009040     MSVCRT:gs_cookie.obj
 0003:00000048       __security_cookie_complement 0000000180009048     MSVCRT:gs_cookie.obj
 0003:00000050       __scrt_native_dllmain_reason 0000000180009050     MSVCRT:utility.obj
 0003:00000058       __isa_available            0000000180009058     MSVCRT:cpu_disp.obj
 0003:0000005c       __isa_enabled              000000018000905c     MSVCRT:cpu_disp.obj
 0003:00000060       __memset_fast_string_threshold 0000000180009060     MSVCRT:cpu_disp.obj
 0003:00000068       __memset_nt_threshold      0000000180009068     MSVCRT:cpu_disp.obj
 0003:00000070       __scrt_ucrt_dll_is_in_use  0000000180009070     MSVCRT:ucrt_stubs.obj
 0003:00000080       g_wrongHeapCallbacks       0000000180009080     libgetsysprops001.obj
 0003:00000100       g_szTagInfo                0000000180009100     libgetsysprops001.obj
 0003:00002040       g_tagFlags                 000000018000b040     libgetsysprops001.obj
 0003:00002428       g_refsToVerifyCnt          000000018000b428     libgetsysprops001.obj
 0003:0000242c       g_fakeUserData             000000018000b42c     libgetsysprops001.obj
 0003:00002430       g_tagVisitCount            000000018000b430     libgetsysprops001.obj
 0003:000033d0       g_refsToVerify             000000018000c3d0     libgetsysprops001.obj
 0003:0001aad0       g_userDataError            0000000180023ad0     libgetsysprops001.obj
 0003:0001ac70       ?_OptionsStorage@?1??__local_stdio_printf_options@@9@4_KA 0000000180023c70     libgetsysprops001.obj
 0003:0001b238       _tls_index                 0000000180024238     MSVCRT:tlssup.obj
 0003:0001b240       __scrt_current_native_startup_state 0000000180024240     MSVCRT:utility.obj
 0003:0001b248       __scrt_native_startup_lock 0000000180024248     MSVCRT:utility.obj
 0003:0001b288       __scrt_debugger_hook_flag  0000000180024288     MSVCRT:utility_desktop.obj
 0003:0001b290       ?__type_info_root_node@@3U__type_info_node@@A 0000000180024290     MSVCRT:tncleanup.obj
 0003:0001b2a0       ?_OptionsStorage@?1??__local_stdio_scanf_options@@9@4_KA 00000001800242a0     MSVCRT:default_local_stdio_options.obj
 0003:0001b2a8       __favor                    00000001800242a8     MSVCRT:cpu_disp.obj
 0003:0001b2b0       __dyn_tls_init_callback    00000001800242b0     <common>

 entry point at        0001:00002b60

 Static symbols

 0000:fffd9000       .debug$S                   0000000180000000     getsysprops001.exp
 0000:fffd9000       .debug$S                   0000000180000000     vcruntime:VCRUNTIME140.dll
 0000:fffd9000       .debug$S                   0000000180000000     vcruntime:VCRUNTIME140.dll
 0000:fffd9000       .debug$S                   0000000180000000     vcruntime:VCRUNTIME140.dll
 0000:fffd9000       .debug$S                   0000000180000000     vcruntime:VCRUNTIME140.dll
 0000:fffd9000       .debug$S                   0000000180000000     vcruntime:VCRUNTIME140.dll
 0000:fffd9000       .debug$S                   0000000180000000     vcruntime:VCRUNTIME140.dll
 0000:fffd9000       .debug$S                   0000000180000000     vcruntime:VCRUNTIME140.dll
 0000:fffd9000       .debug$S                   0000000180000000     ucrt:api-ms-win-crt-convert-l1-1-0.dll
 0000:fffd9000       .debug$S                   0000000180000000     ucrt:api-ms-win-crt-heap-l1-1-0.dll
 0000:fffd9000       .debug$S                   0000000180000000     ucrt:api-ms-win-crt-heap-l1-1-0.dll
 0000:fffd9000       .debug$S                   0000000180000000     ucrt:api-ms-win-crt-heap-l1-1-0.dll
 0000:fffd9000       .debug$S                   0000000180000000     ucrt:api-ms-win-crt-heap-l1-1-0.dll
 0000:fffd9000       .debug$S                   0000000180000000     ucrt:api-ms-win-crt-runtime-l1-1-0.dll
 0000:fffd9000       .debug$S                   0000000180000000     ucrt:api-ms-win-crt-runtime-l1-1-0.dll
 0000:fffd9000       .debug$S                   0000000180000000     ucrt:api-ms-win-crt-runtime-l1-1-0.dll
 0000:fffd9000       .debug$S                   0000000180000000     ucrt:api-ms-win-crt-runtime-l1-1-0.dll
 0000:fffd9000       .debug$S                   0000000180000000     ucrt:api-ms-win-crt-runtime-l1-1-0.dll
 0000:fffd9000       .debug$S                   0000000180000000     ucrt:api-ms-win-crt-runtime-l1-1-0.dll
 0000:fffd9000       .debug$S                   0000000180000000     ucrt:api-ms-win-crt-runtime-l1-1-0.dll
 0000:fffd9000       .debug$S                   0000000180000000     ucrt:api-ms-win-crt-runtime-l1-1-0.dll
 0000:fffd9000       .debug$S                   0000000180000000     ucrt:api-ms-win-crt-runtime-l1-1-0.dll
 0000:fffd9000       .debug$S                   0000000180000000     ucrt:api-ms-win-crt-runtime-l1-1-0.dll
 0000:fffd9000       .debug$S                   0000000180000000     ucrt:api-ms-win-crt-runtime-l1-1-0.dll
 0000:fffd9000       .debug$S                   0000000180000000     ucrt:api-ms-win-crt-runtime-l1-1-0.dll
 0000:fffd9000       .debug$S                   0000000180000000     ucrt:api-ms-win-crt-runtime-l1-1-0.dll
 0000:fffd9000       .debug$S                   0000000180000000     ucrt:api-ms-win-crt-runtime-l1-1-0.dll
 0000:fffd9000       .debug$S                   0000000180000000     ucrt:api-ms-win-crt-runtime-l1-1-0.dll
 0000:fffd9000       .debug$S                   0000000180000000     ucrt:api-ms-win-crt-runtime-l1-1-0.dll
 0000:fffd9000       .debug$S                   0000000180000000     ucrt:api-ms-win-crt-stdio-l1-1-0.dll
 0000:fffd9000       .debug$S                   0000000180000000     ucrt:api-ms-win-crt-stdio-l1-1-0.dll
 0000:fffd9000       .debug$S                   0000000180000000     ucrt:api-ms-win-crt-stdio-l1-1-0.dll
 0000:fffd9000       .debug$S                   0000000180000000     ucrt:api-ms-win-crt-stdio-l1-1-0.dll
 0000:fffd9000       .debug$S                   0000000180000000     ucrt:api-ms-win-crt-stdio-l1-1-0.dll
 0000:fffd9000       .debug$S                   0000000180000000     ucrt:api-ms-win-crt-stdio-l1-1-0.dll
 0000:fffd9000       .debug$S                   0000000180000000     ucrt:api-ms-win-crt-stdio-l1-1-0.dll
 0000:fffd9000       .debug$S                   0000000180000000     ucrt:api-ms-win-crt-stdio-l1-1-0.dll
 0000:fffd9000       .debug$S                   0000000180000000     ucrt:api-ms-win-crt-stdio-l1-1-0.dll
 0000:fffd9000       .debug$S                   0000000180000000     ucrt:api-ms-win-crt-stdio-l1-1-0.dll
 0000:fffd9000       .debug$S                   0000000180000000     ucrt:api-ms-win-crt-string-l1-1-0.dll
 0000:fffd9000       .debug$S                   0000000180000000     ucrt:api-ms-win-crt-string-l1-1-0.dll
 0000:fffd9000       .debug$S                   0000000180000000     ucrt:api-ms-win-crt-string-l1-1-0.dll
 0000:fffd9000       .debug$S                   0000000180000000     ucrt:api-ms-win-crt-string-l1-1-0.dll
 0000:fffd9000       .debug$S                   0000000180000000     ucrt:api-ms-win-crt-string-l1-1-0.dll
 0000:fffd9000       .debug$S                   0000000180000000     ucrt:api-ms-win-crt-string-l1-1-0.dll
 0000:fffd9000       .debug$S                   0000000180000000     ucrt:api-ms-win-crt-string-l1-1-0.dll
 0000:fffd9000       .debug$S                   0000000180000000     ucrt:api-ms-win-crt-string-l1-1-0.dll
 0000:fffd9000       .debug$S                   0000000180000000     kernel32:KERNEL32.dll
 0000:fffd9000       .debug$S                   0000000180000000     kernel32:KERNEL32.dll
 0000:fffd9000       .debug$S                   0000000180000000     kernel32:KERNEL32.dll
 0000:fffd9000       .debug$S                   0000000180000000     kernel32:KERNEL32.dll
 0000:fffd9000       .debug$S                   0000000180000000     kernel32:KERNEL32.dll
 0000:fffd9000       .debug$S                   0000000180000000     kernel32:KERNEL32.dll
 0000:fffd9000       .debug$S                   0000000180000000     kernel32:KERNEL32.dll
 0000:fffd9000       .debug$S                   0000000180000000     kernel32:KERNEL32.dll
 0000:fffd9000       .debug$S                   0000000180000000     kernel32:KERNEL32.dll
 0000:fffd9000       .debug$S                   0000000180000000     kernel32:KERNEL32.dll
 0000:fffd9000       .debug$S                   0000000180000000     kernel32:KERNEL32.dll
 0000:fffd9000       .debug$S                   0000000180000000     kernel32:KERNEL32.dll
 0000:fffd9000       .debug$S                   0000000180000000     kernel32:KERNEL32.dll
 0000:fffd9000       .debug$S                   0000000180000000     kernel32:KERNEL32.dll
 0000:fffd9000       .debug$S                   0000000180000000     kernel32:KERNEL32.dll
 0000:fffd9000       .debug$S                   0000000180000000     kernel32:KERNEL32.dll
 0000:fffd9000       .debug$S                   0000000180000000     kernel32:KERNEL32.dll
 0000:fffd9000       .debug$S                   0000000180000000     kernel32:KERNEL32.dll
 0000:fffd9000       .debug$S                   0000000180000000     kernel32:KERNEL32.dll
 0000:fffd9000       .debug$S                   0000000180000000     kernel32:KERNEL32.dll
 0000:fffd9000       .debug$S                   0000000180000000     kernel32:KERNEL32.dll
 0000:fffd9000       .debug$S                   0000000180000000     kernel32:KERNEL32.dll
 0000:fffd9000       .debug$S                   0000000180000000     kernel32:KERNEL32.dll
 0000:fffd9000       .debug$S                   0000000180000000     kernel32:KERNEL32.dll
 0000:fffd9000       .debug$S                   0000000180000000     kernel32:KERNEL32.dll
 0000:fffd9000       .debug$S                   0000000180000000     kernel32:KERNEL32.dll
 0000:fffd9000       .debug$S                   0000000180000000     kernel32:KERNEL32.dll
 0000:fffd9000       .debug$S                   0000000180000000     kernel32:KERNEL32.dll
 0001:00000dcc       addRefToVerify             0000000180001dcc f   libgetsysprops001.obj
 0001:00000e40       agentProc                  0000000180001e40 f   libgetsysprops001.obj
 0001:00000ed0       agentThreadWrapper         0000000180001ed0 f   libgetsysprops001.obj
 0001:00001024       checkProperties            0000000180002024 f   libgetsysprops001.obj
 0001:000012a4       check_option               00000001800022a4 f   libgetsysprops001.obj
 0001:000014ec       file_basename              00000001800024ec f   libgetsysprops001.obj
 0001:00002068       startAgentThreadWrapper    0000000180003068 f   libgetsysprops001.obj
 0001:00002394       syncDebuggeeStatus         0000000180003394 f   libgetsysprops001.obj
 0001:0000261c       capture_previous_context   000000018000361c f   MSVCRT:gs_report.obj
 0001:00002690       ?__scrt_initialize_thread_safe_statics@@YAHXZ 0000000180003690 f   MSVCRT:thread_safe_statics.obj
 0001:00002760       ?__scrt_uninitialize_thread_safe_statics@@YAXXZ 0000000180003760 f   MSVCRT:thread_safe_statics.obj
 0001:00002810       $$000000                   0000000180003810     MSVCRT:amdsecgs.obj
 0001:00002840       ?dllmain_crt_dispatch@@YAHQEAUHINSTANCE__@@KQEAX@Z 0000000180003840 f   MSVCRT:dll_dllmain.obj
 0001:00002890       ?dllmain_crt_process_attach@@YAHQEAUHINSTANCE__@@QEAX@Z 0000000180003890 f   MSVCRT:dll_dllmain.obj
 0001:000029a8       ?dllmain_crt_process_detach@@YAH_N@Z 00000001800039a8 f   MSVCRT:dll_dllmain.obj
 0001:00002a2c       ?dllmain_dispatch@@YAHQEAUHINSTANCE__@@KQEAX@Z 0000000180003a2c f   MSVCRT:dll_dllmain.obj
 0001:00003440       $$000000                   0000000180004440     MSVCRT:guard_dispatch.obj
 0001:00003460       $$000000                   0000000180004460     MSVCRT:guard_xfg_dispatch.obj
 0001:00003476       ?fin$0@?0??dllmain_crt_process_attach@@YAHQEAUHINSTANCE__@@QEAX@Z@4HA 0000000180004476 f   MSVCRT:dll_dllmain.obj
 0001:0000348d       ?fin$0@?0??dllmain_crt_process_detach@@YAH_N@Z@4HA 000000018000448d f   MSVCRT:dll_dllmain.obj
 0001:000034a6       ?fin$1@?0??dllmain_crt_process_detach@@YAH_N@Z@4HA 00000001800044a6 f   MSVCRT:dll_dllmain.obj
 0001:000034ba       ?filt$0@?0??dllmain_dispatch@@YAHQEAUHINSTANCE__@@KQEAX@Z@4HA 00000001800044ba f   MSVCRT:dll_dllmain.obj
 0001:000034f0       __scrt_is_nonwritable_in_current_image$filt$0 00000001800044f0 f   MSVCRT:utility.obj
 0002:00000218       ?__scrt_initialize_tss_var@@3P6AHXZEA 0000000180005218     MSVCRT:thread_safe_statics.obj
 0002:00000340       ?opcLengths@@3QBEB         0000000180005340     libgetsysprops001.obj
 0002:00002000       GS_ExceptionPointers       0000000180007000     MSVCRT:gs_report.obj
 0002:000026d8       $unwind$fprintf            00000001800076d8     libgetsysprops001.obj
 0002:000026e4       $unwind$printf             00000001800076e4     libgetsysprops001.obj
 0002:000026f0       $unwind$?NewObject@JNIEnv_@@QEAAPEAV_jobject@@PEAV_jclass@@PEAU_jmethodID@@ZZ 00000001800076f0     libgetsysprops001.obj
 0002:000026f0       $unwind$nsk_lcomplain      00000001800076f0     libgetsysprops001.obj
 0002:000026f0       $unwind$nsk_ldisplay       00000001800076f0     libgetsysprops001.obj
 0002:000026f8       $unwind$nsk_lvdisplay      00000001800076f8     libgetsysprops001.obj
 0002:000026f8       $unwind$_RTC_Initialize    00000001800076f8     MSVCRT:initsect.obj
 0002:000026f8       $unwind$_RTC_Terminate     00000001800076f8     MSVCRT:initsect.obj
 0002:000026f8       $unwind$?__scrt_initialize_thread_safe_statics@@YAHXZ 00000001800076f8     MSVCRT:thread_safe_statics.obj
 0002:00002704       $unwind$nsk_complain       0000000180007704     libgetsysprops001.obj
 0002:00002704       $unwind$nsk_printf         0000000180007704     libgetsysprops001.obj
 0002:0000270c       $unwind$nsk_lvcomplain     000000018000770c     libgetsysprops001.obj
 0002:00002724       $unwind$nsk_ltrace         0000000180007724     libgetsysprops001.obj
 0002:00002724       $unwind$__report_gsfailure 0000000180007724     MSVCRT:gs_report.obj
 0002:0000272c       $unwind$agentProc          000000018000772c     libgetsysprops001.obj
 0002:0000272c       $unwind$nsk_lvtrace        000000018000772c     libgetsysprops001.obj
 0002:0000272c       $unwind$__raise_securityfailure 000000018000772c     MSVCRT:gs_report.obj
 0002:0000272c       $unwind$__scrt_initialize_crt 000000018000772c     MSVCRT:utility.obj
 0002:0000272c       $unwind$__scrt_initialize_onexit_tables 000000018000772c     MSVCRT:utility.obj
 0002:0000272c       $unwind$__scrt_release_startup_lock 000000018000772c     MSVCRT:utility.obj
 0002:0000272c       $unwind$__scrt_uninitialize_crt 000000018000772c     MSVCRT:utility.obj
 0002:0000272c       $unwind$_onexit            000000018000772c     MSVCRT:utility.obj
 0002:00002734       $unwind$nsk_lverify        0000000180007734     libgetsysprops001.obj
 0002:00002744       $unwind$nsk_vprintf        0000000180007744     libgetsysprops001.obj
 0002:00002754       $unwind$?nsk_jni_lverify@@YAHHPEAUJNIEnv_@@HQEBDH1ZZ 0000000180007754     libgetsysprops001.obj
 0002:00002768       $unwind$?nsk_jni_check_exception@@YAHPEAUJNIEnv_@@QEBDH@Z 0000000180007768     libgetsysprops001.obj
 0002:00002784       $unwind$nsk_jvmti_parseOptions 0000000180007784     libgetsysprops001.obj
 0002:000027a0       $unwind$nsk_jvmti_createJVMTIEnv 00000001800077a0     libgetsysprops001.obj
 0002:000027b4       $unwind$check_option       00000001800077b4     libgetsysprops001.obj
 0002:000027b4       $unwind$nsk_jvmti_waitForSync 00000001800077b4     libgetsysprops001.obj
 0002:000027b4       $unwind$_DllMainCRTStartup 00000001800077b4     MSVCRT:dll_dllmain.obj
 0002:000027c4       $unwind$Java_nsk_jvmti_unit_FollowReferences_FollowRefObjects_resetTags 00000001800077c4     libgetsysprops001.obj
 0002:000027c4       $unwind$addRefToVerify     00000001800077c4     libgetsysprops001.obj
 0002:000027c4       $unwind$nsk_jvmti_resetAgentData 00000001800077c4     libgetsysprops001.obj
 0002:000027c4       $unwind$nsk_jvmti_resumeSync 00000001800077c4     libgetsysprops001.obj
 0002:000027c4       $unwind$__scrt_initialize_default_local_stdio_options 00000001800077c4     MSVCRT:default_local_stdio_options.obj
 0002:000027c4       $unwind$?dllmain_crt_dispatch@@YAHQEAUHINSTANCE__@@KQEAX@Z 00000001800077c4     MSVCRT:dll_dllmain.obj
 0002:000027c4       $unwind$DllMain            00000001800077c4     MSVCRT:dll_dllmain_stub.obj
 0002:000027c4       $unwind$__GSHandlerCheck   00000001800077c4     MSVCRT:gshandler.obj
 0002:000027c4       $unwind$?__scrt_uninitialize_thread_safe_statics@@YAXXZ 00000001800077c4     MSVCRT:thread_safe_statics.obj
 0002:000027c4       $unwind$__scrt_acquire_startup_lock 00000001800077c4     MSVCRT:utility.obj
 0002:000027c4       $unwind$__scrt_dllmain_after_initialize_c 00000001800077c4     MSVCRT:utility.obj
 0002:000027c4       $unwind$__scrt_dllmain_before_initialize_c 00000001800077c4     MSVCRT:utility.obj
 0002:000027c4       $unwind$__scrt_dllmain_crt_thread_attach 00000001800077c4     MSVCRT:utility.obj
 0002:000027c4       $unwind$__scrt_dllmain_crt_thread_detach 00000001800077c4     MSVCRT:utility.obj
 0002:000027c4       $unwind$__scrt_dllmain_uninitialize_c 00000001800077c4     MSVCRT:utility.obj
 0002:000027c4       $unwind$__scrt_dllmain_uninitialize_critical 00000001800077c4     MSVCRT:utility.obj
 0002:000027c4       $unwind$atexit             00000001800077c4     MSVCRT:utility.obj
 0002:000027cc       $unwind$nsk_jvmti_lverify  00000001800077cc     libgetsysprops001.obj
 0002:000027e0       $unwind$exitOnError        00000001800077e0     libgetsysprops001.obj
 0002:000027f0       $unwind$Java_nsk_share_jvmti_ArgumentHandler_getAgentOptionsString 00000001800077f0     libgetsysprops001.obj
 0002:00002804       $unwind$Java_nsk_jvmti_unit_FollowReferences_FollowRefObjects_getTag 0000000180007804     libgetsysprops001.obj
 0002:00002804       $unwind$Java_nsk_share_jvmti_DebugeeClass_checkStatus 0000000180007804     libgetsysprops001.obj
 0002:00002804       $unwind$agentThreadWrapper 0000000180007804     libgetsysprops001.obj
 0002:00002814       $unwind$startAgentThreadWrapper 0000000180007814     libgetsysprops001.obj
 0002:00002830       $unwind$syncDebuggeeStatus 0000000180007830     libgetsysprops001.obj
 0002:00002830       $unwind$__scrt_dllmain_exception_filter 0000000180007830     MSVCRT:utility.obj
 0002:00002844       $unwind$Java_nsk_share_jvmti_DebugeeClass_resetAgentData 0000000180007844     libgetsysprops001.obj
 0002:0000284c       $unwind$MA_checkStatus     000000018000784c     libgetsysprops001.obj
 0002:00002860       $unwind$Java_nsk_jvmti_unit_FollowReferences_FollowRefObjects_setTag 0000000180007860     libgetsysprops001.obj
 0002:00002878       $unwind$Java_nsk_jvmti_unit_FollowReferences_FollowRefObjects_addRefToVerify 0000000180007878     libgetsysprops001.obj
 0002:00002894       $unwind$Agent_Initialize   0000000180007894     libgetsysprops001.obj
 0002:000028ac       $unwind$checkProperties    00000001800078ac     libgetsysprops001.obj
 0002:000028c4       $unwind$capture_previous_context 00000001800078c4     MSVCRT:gs_report.obj
 0002:000028d0       $unwind$__GSHandlerCheckCommon 00000001800078d0     MSVCRT:gshandler.obj
 0002:000028d8       $xdatasym                  00000001800078d8     MSVCRT:amdsecgs.obj
 0002:000028dc       $unwind$?dllmain_crt_process_attach@@YAHQEAUHINSTANCE__@@QEAX@Z 00000001800078dc     MSVCRT:dll_dllmain.obj
 0002:00002918       $unwind$?fin$0@?0??dllmain_crt_process_attach@@YAHQEAUHINSTANCE__@@QEAX@Z@4HA 0000000180007918     MSVCRT:dll_dllmain.obj
 0002:00002918       $unwind$?fin$0@?0??dllmain_crt_process_detach@@YAH_N@Z@4HA 0000000180007918     MSVCRT:dll_dllmain.obj
 0002:00002918       $unwind$?fin$1@?0??dllmain_crt_process_detach@@YAH_N@Z@4HA 0000000180007918     MSVCRT:dll_dllmain.obj
 0002:00002920       $unwind$?dllmain_crt_process_detach@@YAH_N@Z 0000000180007920     MSVCRT:dll_dllmain.obj
 0002:00002974       $unwind$?dllmain_dispatch@@YAHQEAUHINSTANCE__@@KQEAX@Z 0000000180007974     MSVCRT:dll_dllmain.obj
 0002:0000299c       $unwind$?filt$0@?0??dllmain_dispatch@@YAHQEAUHINSTANCE__@@KQEAX@Z@4HA 000000018000799c     MSVCRT:dll_dllmain.obj
 0002:000029a4       $unwind$__scrt_is_nonwritable_in_current_image 00000001800079a4     MSVCRT:utility.obj
 0002:000029c4       $unwind$__scrt_is_nonwritable_in_current_image$filt$0 00000001800079c4     MSVCRT:utility.obj
 0002:000029cc       $unwind$__scrt_fastfail    00000001800079cc     MSVCRT:utility_desktop.obj
 0002:000029dc       $unwind$__security_init_cookie 00000001800079dc     MSVCRT:gs_support.obj
 0002:000029e8       $unwind$__isa_available_init 00000001800079e8     MSVCRT:cpu_disp.obj
 0002:000029f8       $xdatasym                  00000001800079f8     MSVCRT:guard_dispatch.obj
 0002:00002a00       $xdatasym                  0000000180007a00     MSVCRT:guard_xfg_dispatch.obj
 0002:00002a10       .edata                     0000000180007a10     getsysprops001.exp
 0002:00002a38       rgpv                       0000000180007a38     getsysprops001.exp
 0002:00002a70       rgszName                   0000000180007a70     getsysprops001.exp
 0002:00002aa8       rgwOrd                     0000000180007aa8     getsysprops001.exp
 0002:00002ac4       szName                     0000000180007ac4     getsysprops001.exp
 0002:00002ad7       $N00001                    0000000180007ad7     getsysprops001.exp
 0002:00002ae6       $N00002                    0000000180007ae6     getsysprops001.exp
 0002:00002af3       $N00003                    0000000180007af3     getsysprops001.exp
 0002:00002b38       $N00004                    0000000180007b38     getsysprops001.exp
 0002:00002b75       $N00005                    0000000180007b75     getsysprops001.exp
 0002:00002bbd       $N00006                    0000000180007bbd     getsysprops001.exp
 0002:00002bfd       $N00007                    0000000180007bfd     getsysprops001.exp
 0002:00002c3a       $N00008                    0000000180007c3a     getsysprops001.exp
 0002:00002c75       $N00009                    0000000180007c75     getsysprops001.exp
 0002:00002ca3       $N00010                    0000000180007ca3     getsysprops001.exp
 0002:00002cd4       $N00011                    0000000180007cd4     getsysprops001.exp
 0002:00002d03       $N00012                    0000000180007d03     getsysprops001.exp
 0002:00002d32       $N00013                    0000000180007d32     getsysprops001.exp
 0002:00002d67       $N00014                    0000000180007d67     getsysprops001.exp
 0002:000031ca       .idata$6                   00000001800081ca     kernel32:KERNEL32.dll
 0002:0000322e       .idata$6                   000000018000822e     vcruntime:VCRUNTIME140.dll
 0002:000033c0       .idata$6                   00000001800083c0     ucrt:api-ms-win-crt-heap-l1-1-0.dll
 0002:000033e0       .idata$6                   00000001800083e0     ucrt:api-ms-win-crt-runtime-l1-1-0.dll
 0002:00003402       .idata$6                   0000000180008402     ucrt:api-ms-win-crt-convert-l1-1-0.dll
 0002:00003424       .idata$6                   0000000180008424     ucrt:api-ms-win-crt-stdio-l1-1-0.dll
 0002:00003444       .idata$6                   0000000180008444     ucrt:api-ms-win-crt-string-l1-1-0.dll
 0003:00000000       ?codeAttributeName@@3PEBDEB 0000000180009000     libgetsysprops001.obj
 0003:00000008       ?lineNumberAttributeName@@3PEBDEB 0000000180009008     libgetsysprops001.obj
 0003:00000010       ?localVarAttributeName@@3PEBDEB 0000000180009010     libgetsysprops001.obj
 0003:00000018       ?localVarTypeAttributeName@@3PEBDEB 0000000180009018     libgetsysprops001.obj
 0003:00000020       ?stackMapAttributeName@@3PEBDEB 0000000180009020     libgetsysprops001.obj
 0003:00000028       ?callBytes@@3PAEA          0000000180009028     libgetsysprops001.obj
 0003:0000002c       ?allocBytes@@3PAEA         000000018000902c     libgetsysprops001.obj
 0003:0001aad4       redefineAttempted          0000000180023ad4     libgetsysprops001.obj
 0003:0001aad8       nsk_context                0000000180023ad8     libgetsysprops001.obj
 0003:0001aae4       redefineSucceed            0000000180023ae4     libgetsysprops001.obj
 0003:0001aae8       agentFailed                0000000180023ae8     libgetsysprops001.obj
 0003:0001aaec       currentAgentStatus         0000000180023aec     libgetsysprops001.obj
 0003:0001aaf0       context                    0000000180023af0     libgetsysprops001.obj
 0003:0001aba8       agentThread                0000000180023ba8     libgetsysprops001.obj
 0003:0001abb0       agentThreadProc            0000000180023bb0     libgetsysprops001.obj
 0003:0001abb8       agentThreadArg             0000000180023bb8     libgetsysprops001.obj
 0003:0001abc0       agent_data                 0000000180023bc0     libgetsysprops001.obj
 0003:0001abd0       jvmti_env                  0000000180023bd0     libgetsysprops001.obj
 0003:0001abd8       jvm                        0000000180023bd8     libgetsysprops001.obj
 0003:0001abe0       jni_env                    0000000180023be0     libgetsysprops001.obj
 0003:0001abe8       checkStatus_func           0000000180023be8     libgetsysprops001.obj
 0003:0001abf0       ?codeAttributeIndex@@3GA   0000000180023bf0     libgetsysprops001.obj
 0003:0001abf4       ?lineNumberAttributeIndex@@3GA 0000000180023bf4     libgetsysprops001.obj
 0003:0001abf8       ?localVarAttributeIndex@@3GA 0000000180023bf8     libgetsysprops001.obj
 0003:0001abfc       ?localVarTypeAttributeIndex@@3GA 0000000180023bfc     libgetsysprops001.obj
 0003:0001ac00       ?stackMapAttributeIndex@@3GA 0000000180023c00     libgetsysprops001.obj
 0003:0001ac04       ?stackFrameOffset@@3GA     0000000180023c04     libgetsysprops001.obj
 0003:0001ac08       ?mode@@3HA                 0000000180023c08     libgetsysprops001.obj
 0003:0001ac0c       ?constantPoolSize@@3GA     0000000180023c0c     libgetsysprops001.obj
 0003:0001ac10       ?orig@@3PEBEEB             0000000180023c10     libgetsysprops001.obj
 0003:0001ac18       ?gen@@3PEAEEA              0000000180023c18     libgetsysprops001.obj
 0003:0001ac20       ?inputPos@@3PEAEEA         0000000180023c20     libgetsysprops001.obj
 0003:0001ac28       ?endPos@@3PEBEEB           0000000180023c28     libgetsysprops001.obj
 0003:0001ac30       ?genPos@@3PEAEEA           0000000180023c30     libgetsysprops001.obj
 0003:0001ac38       ?markPos@@3PEAEEA          0000000180023c38     libgetsysprops001.obj
 0003:0001ac40       ?constantPool@@3PEAPEADEA  0000000180023c40     libgetsysprops001.obj
 0003:0001ac48       ?constantPoolCount@@3GA    0000000180023c48     libgetsysprops001.obj
 0003:0001ac4c       ?zeroBytes@@3PAEA          0000000180023c4c     libgetsysprops001.obj
 0003:0001ac50       ?codeLength@@3IA           0000000180023c50     libgetsysprops001.obj
 0003:0001ac58       ?map@@3PEAIEA              0000000180023c58     libgetsysprops001.obj
 0003:0001ac60       ?widening@@3PEACEA         0000000180023c60     libgetsysprops001.obj
 0003:0001ac68       timeout                    0000000180023c68     libgetsysprops001.obj
 0003:0001ac80       GS_ExceptionRecord         0000000180023c80     MSVCRT:gs_report.obj
 0003:0001ad20       GS_ContextRecord           0000000180023d20     MSVCRT:gs_report.obj
 0003:0001b1f0       ?g_tss_cv@@3U_RTL_CONDITION_VARIABLE@@A 00000001800241f0     MSVCRT:thread_safe_statics.obj
 0003:0001b1f8       ?g_tss_event@@3PEAXEA      00000001800241f8     MSVCRT:thread_safe_statics.obj
 0003:0001b200       ?g_tss_mutex@@3U_RTL_CRITICAL_SECTION@@A 0000000180024200     MSVCRT:thread_safe_statics.obj
 0003:0001b228       ?g_sleep_condition_variable_cs@@3P6AHPEAU_RTL_CONDITION_VARIABLE@@PEAU_RTL_CRITICAL_SECTION@@K@ZEA 0000000180024228     MSVCRT:thread_safe_statics.obj
 0003:0001b230       ?g_wake_all_condition_variable@@3P6AXPEAU_RTL_CONDITION_VARIABLE@@@ZEA 0000000180024230     MSVCRT:thread_safe_statics.obj
 0003:0001b23c       ?__proc_attached@@3HA      000000018002423c     MSVCRT:dll_dllmain.obj
 0003:0001b250       ?is_initialized_as_dll@@3_NA 0000000180024250     MSVCRT:utility.obj
 0003:0001b251       ?module_local_atexit_table_initialized@@3_NA 0000000180024251     MSVCRT:utility.obj
 0003:0001b258       ?module_local_atexit_table@@3U_onexit_table_t@@A 0000000180024258     MSVCRT:utility.obj
 0003:0001b270       ?module_local_at_quick_exit_table@@3U_onexit_table_t@@A 0000000180024270     MSVCRT:utility.obj
